:100000000C94AA000C942D020C94C7000C94C70009
:100010000C94C7000C94C7000C94C7000C94C70044
:100020000C94C7000C94C7000C94C7000C94C70034
:100030000C94C7000C94C7000C94C7000C94C70024
:100040000C94C7000C94C7000C94C7000C94C70014
:100050000C94C7000C94C7000C94C7000C94C70004
:100060000C94C7000C94C700040309041803720021
:100070006100700068006E00650074002E006E0064
:10008000650074000A0331003000300030000501C3
:100090000904A1010901A1008501093009311500F8
:1000A00026FF007508950281020509190129081526
:1000B000002501750195088102C0C005010904A150
:1000C000010901A100850209300931150026FF0050
:1000D00075089502810205091901290815002501F5
:1000E000750195088102C0C005010904A10109013B
:1000F000A100850309300931150026FF0075089518
:1001000002810205091901290815002501750195CB
:10011000088102C0C005010904A1010901A10085EF
:100120000409300931150026FF0075089502810287
:100130000509190129081500250175019508810295
:10014000C0C012010101000000089B280300040147
:100150000102030111241FBECFEFD4E0DEBFCDBFEB
:1001600011E0A0E0B1E0E8EEFEE002C005900D92E3
:10017000AC34B107D9F711E0ACE4B1E001C01D9295
:10018000AB3AB107E1F70E94DE030C9472070C94BE
:100190000000E9E6F0E0808183608083E89A83ECE8
:1001A0008093810108950F931F93CF93DF939091D4
:1001B000910119160CF0B3C020918E0180918D0130
:1001C0008D3209F0A2C08AE5809301019B3009F0CD
:1001D0009CC0CCE0D0E0C21BD109CB56DE4F888159
:1001E000807609F083C010927F018981882359F4B9
:1001F000109280018FE791E09093900180938F019E
:1002000030E822E07BC0853021F48A81809392011E
:100210006BC0863009F04DC08B81813009F443C03A
:10022000823021F4CE010E94900363C0833071F5C7
:100230008A81882349F488E690E090939001809326
:100240008F0130EC24E05AC0813049F48CE690E014
:100250009093900180938F0130EC28E14FC0823061
:1002600049F483E091E09093900180938F0130E80E
:1002700026E144C0833009F03FC084E890E09093C9
:10028000900180938F0130EC2CE038C0813249F42A
:100290008FE591E09093900180938F0130EC29E0FD
:1002A0002DC0823249F5CE010E949003282F30ECF8
:1002B00025C0883019F484E991E00AC0893021F41E
:1002C0008A818093940110C08A3049F48FE791E0CD
:1002D0009093900180938F0130E821E00FC08B3024
:1002E00019F483EC8093810130E807C0CE010E94AD
:1002F000BE03282F30E802C030EC20E08F81882335
:1003000039F48E81821728F003C030E880E001C004
:10031000822F30934C0180930001109291018091C3
:10032000010184FF4AC0809100018F3F09F445C05C
:10033000182F893008F018E0811B8093000180910C
:100340004C0180FD02C00BE401C003EC8F5F809381
:100350004C0120918F013091900186FD05C0D9019B
:10036000912FE7E7F1E011C0A7E7B1E080E090E06E
:1003700006C0F901E80FF91FE491ED9301961817F3
:10038000C1F705C08D91819391509923D9F7F90157
:10039000E10FF11DF0939001E0938F0187E791E069
:1003A000612F0E942902183019F08FEF809300010D
:1003B000009376011C5F109301019AE089B185706A
:1003C00031F49150D9F71092920110928C01DF9183
:1003D000CF911F910F9108951F93DC01162F8091EB
:1003E000020184FF0AC08091810198E889278093E7
:1003F0008101912FE2E8F1E007C08AE580930201D4
:10040000F8CF8D91819391509923D9F782E891E0AB
:10041000612F0E9429021C5F109302011F91089511
:10042000A82FB92F8FEF9FEF41E050EA615070F095
:100430002D9138E0722F782796958795269570FF35
:1004400002C0842795273A95A9F7F0CF809590951B
:100450000895E6DF8D939D930895CF93CFB7CF9303
:10046000489BFECF489B09C0489B07C0489B05C0DE
:10047000489B03C0489B01C09EC0DF93C0918E0182
:10048000DD27CB56DE4F489B02C0DF91EBCF2F9389
:100490000F931F9309B12FEF00FB20F94F933F9368
:1004A00019B14FEF012700FB21F93BE031C04E7F2E
:1004B000012F19B1216028C0102F4D7F226000004C
:1004C00009B129C04B7F2460012F000019B12BC056
:1004D00019B1477F28602AC04F7E09B120612CC026
:1004E0004F7D19B120622FC04F7B09B1206432C00B
:1004F000422709B149934FEF0000102710FB20F964
:1005000019B11570A9F1297F91F2012700FB21F99A
:1005100009B1237F89F23150F0F1102710FB22F945
:1005200019B1277E79F2012700FB23F92F7C81F294
:1005300009B1102710FB24F92F7971F200C019B10D
:10054000012700FB25F92F7359F200C009B11027CC
:1005500010FB26F9223040F200C019B1012700FB40
:1005600027F9243028F64F77206819B10000F9CF19
:100570003B503195333011E01CBBB8F0C31BD04069
:100580000881033C41F10B3431F11981412F1F7770
:1005900020918C01121731F4093691F10D3279F066
:1005A000013E69F02227209393013F914F911F91C3
:1005B0000F912F91DF91CF91CFBFCF9118950093DD
:1005C00093013F914F911F910F912F91DF91CCB3E8
:1005D000C0FD46CFF0CF00919301002331F310917D
:1005E00091011123A1F53430A2F1309391010093D0
:1005F0008D0110918E013BE0311B30938E0129C09B
:100600000091910101301CF50AE547FD09C03091C8
:10061000010134FD20C000930101C6E7D1E01FC0F5
:100620003091020134FD17C000930201C1E8D1E00E
:1006300016C0052710E00BB91FC0052722C00527EB
:1006400027C005272CC0052710E00BB933C04AE5A9
:1006500003C042ED01C0432FC4E1D0E032E01AB143
:100660001560589A0BB11AB95F9355E020E820FF46
:1006700005270BB9279517951C3FD8F620FF0527AE
:1006800027950BB917951C3FC0F620FF0527279526
:1006900017950BB91C3F98F620FF0527279517954E
:1006A0001C3F0BB970F600C0499120FF05270BB91C
:1006B000279517951C3F38F620FF052727950BB97E
:1006C00017951C3F38F520FF0527279517950BB97F
:1006D0001C3F10F520FF0527279517951C3F0BB9E8
:1006E000E8F4242F3A9519F60A7F5F910BB900C000
:1006F00010919201C651D04011F010938C0111E07D
:100700001CBB01601AB11A7F402F4A7F0BB91AB97E
:100710004BB94BCF0527D3CF0527D8CF0527DDCF42
:10072000FC018081807641F58181863029F58381C5
:100730008230D1F0823269F08130F1F48091510140
:10074000909152019093900180938F018091530179
:10075000089580914E0190914F0190939001809364
:100760008F0180915001089587E191E0909390016D
:1007700080938F0182E2089580E00895DC0127E5EF
:1007800031E03093900120938F018C9180768032FC
:1007900099F411968C911197813071F41092540153
:1007A000E0915501F09156010784F089E02DC901CF
:1007B00012966C910995089580E00895DF92EF926A
:1007C000FF920F931F93CF93DF9381E084B98EEF55
:1007D00085B917B88FEF88B988EF8BB985E08AB9EA
:1007E00082E08093B00087E08093B10084EC809336
:1007F000B30080E395E70197F1F783B190E086704D
:10080000907095958795823011F40E94BD040E94E6
:100810009906FC0190935601809355018381948140
:1008200090934F0180934E01818180935001878185
:100830009085009731F0909352018093510185810A
:1008400008C082E491E090935201809351010E948C
:1008500062078093530180915001809330018BB1E6
:100860008A7F8BB98AB185608AB988EC9FEA019743
:10087000F1F78AB18A7F8AB9E0915501F09156016A
:100880000184F285E02D09950E94C900E09155018F
:10089000F09156010384F485E02D0995789492E057
:1008A000D92E81E0E82EF12CA8950E94D300B99BA7
:1008B000FBCFD7BAE0915501F09156010384F4853E
:1008C000E02D099510E0C0E0D0E012C00584F68567
:1008D000E02D9E012F5F822F0995882341F0C701EB
:1008E0000C2E02C0880F991F0A94E2F7182B21964C
:1008F000E0915501F09156018081992787FD9095EF
:10090000C817D9071CF3112379F2C0E0D0E0012FFA
:10091000112707FD109524C0C8010C2E02C0959523
:1009200087950A94E2F780FF1AC08091020184FF44
:1009300016C0CE018F5F682F0784F089E02D87E510
:1009400091E00995682F87E591E00E94EC0103C0D2
:100950000E94D300A8958091020184FFF9CF2196CF
:10096000E0915501F09156018081992787FD90957E
:10097000C817D9070CF098CFCFCF10924A0108952D
:1009800080916301882309F44DC0449A80E38A95DD
:10099000F1F7449860E070E020E030E098E1892FC2
:1009A0008A95F1F74598660F770F339B6160329B0C
:1009B0007160892F8A95F1F7459A2F5F3F4F283054
:1009C000310569F740E050E020E030E098E1892F00
:1009D0008A95F1F74598440F550F339B4160329B40
:1009E0005160892F8A95F1F7459A2F5F3F4F283044
:1009F000310569F780E090E038E1232F2A95F1F77F
:100A00004598232F2A95F1F7459A0196883091054C
:100A1000A1F760936601709367014093680150935A
:100A20006901089580916501882309F475C0449A8D
:100A300080E3982F9A95F1F744988A95F1F72D9ACB
:100A400088E18A95F1F720E030E050E060E098E13D
:100A50004598892F8A95F1F7550F660F339B5160A2
:100A6000329B6160459A892F8A95F1F72F5F3F4F3E
:100A70002830310569F7509366016093680120E0E2
:100A800030E098E14598892F8A95F1F7569566955B
:100A9000339B5068329B6068459A892F8A95F1F79D
:100AA0002F5F3F4F2830310569F72D9888E18A95EF
:100AB000F1F720E030E090E040E078E14598872FC2
:100AC0008A95F1F7990F440F339B9160329B4160F7
:100AD000459A872F8A95F1F72F5F3F4F28303105D0
:100AE00069F790936A0140936C0120E030E078E16F
:100AF0004598872F8A95F1F796954695339B906890
:100B0000329B4068459A872F8A95F1F72F5F3F4FB8
:100B10002830310569F749C0449A80E38A95F1F796
:100B2000449820E030E050E060E090E040E078E180
:100B3000872F8A95F1F74598550F660F990F440F47
:100B4000339B5160329B6160319B9160309B41606F
:100B5000872F8A95F1F7459A2F5F3F4F283031054F
:100B600039F7509366016093680190936A0140934E
:100B70006C0120E030E078E1872F8A95F1F7459805
:100B80005695669596954695339B5068329B60685E
:100B9000319B9068309B4068872F8A95F1F7459A82
:100BA0002F5F3F4F2830310539F780914A01882364
:100BB00021F1809164015F3F11F4816001C08E7F5B
:100BC00080936401809164016F3F11F4826001C0E1
:100BD0008D7F80936401809164019F3F11F4846054
:100BE00001C08B7F80936401809164014F3F11F4B9
:100BF000886001C0877F809364018091640180FDDB
:100C000050E05093670181FD60E06093690182FDCF
:100C100090E090936B0183FD40E040936D01089557
:100C20001F931FB7F8943C9A3D9A87B1807F87B98C
:100C300088B18F6088B9459A4498259A2D9A109268
:100C400064010E94C00480914A01882321F58091AB
:100C500067018F3F29F48091640181608093640172
:100C6000809169018F3F29F48091640182608093B3
:100C7000640180916B018F3F29F48091640184604D
:100C80008093640180916D018F3F29F4809164010C
:100C9000886080936401449A80E38A95F1F74498D0
:100CA00080E090E030E040E058E1252F2A95F1F710
:100CB0004598339905C08331910519F441E001C08D
:100CC0003F5F252F2A95F1F7459A019688319105C6
:100CD00061F7442329F0373119F481E080936301EF
:100CE0002D98329B10C0449A90E3892F8A95F1F792
:100CF000329909C04498892F8A95F1F7329B03C035
:100D000081E0809365012D9A329B10C0449A90E354
:100D1000892F8A95F1F7329909C04498892F8A95CD
:100D2000F1F7329B03C081E0809365011FBF1F91E3
:100D300008958EE890E090933D0180933C0189E313
:100D400091E00895CF93DF93EC01653010F080E0DF
:100D500094C080916301E62FFF27E7FDF09588237B
:100D600059F1DF0111972097F9F06883FD01EA59E5
:100D7000FE4F808180FD02C090E801C09FEF81FDA1
:100D800090E09983FD01EA59FE4F808182FD02C007
:100D900090E801C09FEF83FD90E09A83FD01EA593E
:100DA000FE4F8081807F8B83FD01EA59FE4F808159
:100DB000A259BE4F8C9360C0DF011197209709F4B0
:100DC0004FC06883BD01660F771FFB01EA59FE4FD4
:100DD000808180FD02C090E801C09FEF81FD90E01E
:100DE0009983FB01EA59FE4F808182FD02C090E8A1
:100DF00001C09FEF83FD90E09A838091640190E0B1
:100E00000A2E02C0959587950A94E2F7FB01EA59EC
:100E1000FE4F80FF03C08081807F21C06081462F0C
:100E200050E09A012074307075E0359527957A95D9
:100E3000E1F7CA018072907033E0959587953A95F5
:100E4000E1F7282B661F6627661F262B407150701E
:100E500055954795242B81818295807F822B8B83AA
:100E6000FD01EE0FFF1FDF01AA59BE4F8D919C912E
:100E7000E259FE4F9183808384E0DF91CF91089502
:100E8000815090916301A82FB0E0992361F020E098
:100E9000FD01E259FE4FAA59BE4F9C9180819817DF
:100EA00079F021E00DC0BD01660F771FCB018A5993
:100EB0009E4F62597E4F42E050E00E946507282F06
:100EC000822F089582E190E00895FB01DC0104C0C7
:100ED0008D910190801921F441505040C8F7881B32
:080EE000990B0895F894FFCF6F
:100EE800FF5A5A140334006E00650073003400730F
:100EF800006E0065007300090222000101008032C3
:100F08000904000001030000000921010100012279
:100F180000000705810308000A04B400000000006F
:0C0F280000001006C0044007A2060100F3
:00000001FF
